:100000000C9434000C9451000C9451000C94510049
:100010000C9451000C9451000C9451000C94E50088
:100020000C9451000C9451000C9451000C94B400A9
:100030000C9451000C9451000C9483000C945100CA
:100040000C9451000C9451000C9451000C945100EC
:100050000C9451000C9451000C9451000C945100DC
:100060000C9451000C94510011241FBECFEFD8E026
:10007000DEBFCDBF11E0A0E0B1E0E8E7F5E002C0EF
:1000800005900D92A431B107D9F711E0A4E1B1E0D8
:1000900001C01D92A931B107E1F70E9433010C9410
:1000A000BA020C9400008230910561F08330910512
:1000B00099F00197C9F416BC80916E00826080931C
:1000C0006E0016C0109285001092840080916F001F
:1000D000826080936F000CC01092B200809170001B
:1000E00082608093700004C081E090E00E94BA02B8
:1000F00078949FB7F894809116019FBF8823C9F325
:100100001092160108951F920F920FB60F921124AC
:100110002F933F938F939F9380911401909115019A
:1001200001969093150180931401809116018130FE
:1001300091F0209114013091150180911701909157
:1001400018012817390738F081E0809316011092C2
:100150001501109214019F918F913F912F910F9053
:100160000FBE0F901F9018951F920F920FB60F920F
:1001700011242F933F938F939F938091140190911B
:100180001501019690931501809314018091160139
:10019000813091F020911401309115018091170167
:1001A000909118012817390738F081E080931601E3
:1001B00010921501109214019F918F913F912F91F0
:1001C0000F900FBE0F901F9018951F920F920FB6B1
:1001D0000F9211242F933F938F939F93809114013B
:1001E00090911501019690931501809314018091CF
:1001F0001601813091F02091140130911501809108
:100200001701909118012817390738F081E0809381
:10021000160110921501109214019F918F913F9138
:100220002F910F900FBE0F901F901895FC012498EE
:1002300083E290E09787868785B5836085BD81E0FE
:1002400090E0918B808B22E030E030931801209376
:10025000170124B5226024BD29EF27BD938B828B23
:1002600080E090E00895CF92DF92EF92FF9280E0DD
:1002700091E00E941601C12CD12C760160E070E063
:10028000CB01609300017093010180930201909370
:10029000030180911201909113010E9453008FEF8E
:1002A000C81AD80AE80AF80AC701B6010E94C901AB
:1002B0002FE632E143E05BE30E94570220E030E0AA
:1002C000A9010E946501DDCF5058BB27AA270ED097
:1002D000B4C0A5D030F0AAD020F031F49F3F11F483
:1002E0001EF49AC00EF4E095E7FB90C0E92FB6D05B
:1002F00080F3BA17620773078407950718F071F443
:100300009EF5CEC00EF4E0950B2EBA2FA02D0B015A
:10031000B90190010C01CA01A0011124FF27591B4A
:1003200099F0593F50F4503E68F11A16F040A22F50
:10033000232F342F4427585FF3CF469537952795C1
:10034000A795F0405395C9F77EF41F16BA0B620BC0
:10035000730B840BBAF09150A1F0FF0FBB1F661F07
:10036000771F881FC2F70EC0BA0F621F731F841F4A
:1003700048F4879577956795B795F7959E3F08F070
:10038000B3CF9395880F08F09927EE0F979587952F
:100390000895E89409C097FB3EF490958095709578
:1003A00061957F4F8F4F9F4F9923A9F0F92F96E9C1
:1003B000BB279395F695879577956795B795F11136
:1003C000F8CFFAF4BB0F11F460FF1BC06F5F7F4FD3
:1003D0008F4F9F4F16C0882311F096E911C07723E5
:1003E00021F09EE8872F762F05C0662371F096E8EE
:1003F000862F70E060E02AF09A95660F771F881FBD
:10040000DAF7880F9695879597F9089597F99F677A
:1004100080E870E060E008959FEF80EC089500248C
:100420000A941616170618060906089500240A9459
:1004300012161306140605060895092E0394000CDF
:1004400011F4882352F0BB0F40F4BF2B11F460FF6E
:1004500004C06F5F7F4F8F4F9F4F089557FD905897
:10046000440F551F59F05F3F71F04795880F97FB78
:10047000991F61F09F3F79F0879508951216130632
:100480001406551FF2CF4695F1DF08C01616170661
:100490001806991FF1CF8695710561050894089596
:1004A000E894BB2766277727CB0197F908950BD0EF
:1004B000C4CFB5DF28F0BADF18F0952309F0A6CF36
:1004C000ABCF1124EECFCADFA0F3959FD1F3950FE8
:1004D00050E0551F629FF001729FBB27F00DB11DC8
:1004E000639FAA27F00DB11DAA1F649F6627B00D58
:1004F000A11D661F829F2227B00DA11D621F739F41
:10050000B00DA11D621F839FA00D611D221F749F4E
:100510003327A00D611D231F849F600D211D822F95
:10052000762F6A2F11249F5750408AF0E1F08823DC
:100530004AF0EE0FFF1FBB1F661F771F881F9150E9
:100540005040A9F79E3F510570F060CFAACF5F3FA2
:10055000ECF3983EDCF3869577956795B795F7951C
:10056000E7959F5FC1F7FE2B880F911D96958795A4
:0805700097F90895F894FFCFFC
:1005780000000000000000006F12033B01000000B3
:04058800000000006F
:00000001FF
